:100000000C942A000C943C000C943C000C943C0092
:100010000C943C000C943C000C943C000C943C0070
:100020000C943C000C9450000C943C000C940D0279
:100030000C9436020C943C000C943C000C943C0054
:100040000C943C000C943C000C943C000C943C0040
:100050000C943C0011241FBECFE5D4E0DEBFCDBF21
:1000600010E0A0E6B0E001C01D92AD3AB107E1F7A3
:100070000E94C2000C94F6020C94000081B38370BD
:1000800081BB82B38C6F82BBB898C09AD79ADF9835
:1000900085E083BF84E682BF89B7816089BF089508
:1000A0001F920F920FB60F9211242F933F934F93ED
:1000B0005F938F939F9384E682BF4091AB005091F2
:1000C000AC0080B396B3392F20E090E0822B932BC5
:1000D0008095909584279527209162003091630048
:1000E00028233923209530953093630020936200B4
:1000F00040916000509161004823592342275327C3
:1001000050936100409360008223932384239523BE
:100110002091AB003091AC00282739273093AC00F8
:100120002093AB002091A9003091AA004091AB0030
:100130005091AC0048235923422B532B5093AA00D3
:100140004093A9009F918F915F914F913F912F9183
:100150000F900FBE0F901F9018959C01F8948091FE
:10016000A9009091AA00282339238091A900909199
:10017000AA00822793279093AA008093A9007894DD
:10018000C90108950E943E000E946C0187E690E03C
:100190000E945B0280E060E00E94B00178940E94BF
:1001A000BD0218161906E4F40E946F028A32910506
:1001B00019F40E94620114C08B32910529F480E089
:1001C00062E00E94B0010CC08732910511F4DF9803
:1001D00007C08332910511F4DF9A02C00E944301E7
:1001E00080E190E00E94AD00009719F086E60E9441
:1001F0008A0280E290E00E94AD00009719F086E448
:100200000E948A0288E090E00E94AD00009719F0F9
:1002100083E70E948A0280E890E00E94AD00009788
:1002200019F081E40E948A0280E490E00E94AD000F
:10023000009719F081E60E948A0280E091E00E9416
:10024000AD00009719F08FE60E948A0284E090E0EA
:100250000E94AD00009709F4A2CF86E70E948A02AF
:100260009ECFDD9A8AE68A95F1F700C0DD98089561
:100270009BB3907F9BBB9BB382958F70892B8BBB6D
:100280000E94310108951F93182FDC9A0E943801B3
:10029000812F8295807F0E94380185EF8A95F1F742
:1002A00000001F9108951F93182FDC980E943801B9
:1002B000812F8295807F0E94380180EE8A95F1F728
:1002C0001F91089581E00E9453018FE39FE1019700
:1002D000F1F700C0000008958AB38F638ABB8BB327
:1002E000807C8BBB8FE59AEE0197F1F700C0000090
:1002F00080E30E9438018FE19EE40197F1F700C08E
:1003000000000E9431018FE99FE00197F1F700C0E2
:1003100000000E9431018FE99FE00197F1F700C0D2
:10032000000080E20E9438018FE19EE40197F1F71E
:1003300000C0000088E20E9453018CE00E9453013B
:1003400086E00E9453010E946201089582E00E94AB
:1003500053018FE39FE10197F1F700C0000008957A
:10036000623061F0633018F4613079F405C06330B5
:1003700039F0643051F406C0805805C0805403C081
:10038000805701C080530E9453010895EF92FF925D
:10039000CF93DF93E82EE7017E01F92EE70102C03B
:1003A0000E94430189918823D9F7DF91CF91FF9073
:1003B000EF900895CF93DF93EC0102C00E944301B8
:1003C000FE01219684918823C9F7DF91CF9108958A
:1003D000EF92FF921F93DF93CF9300D0CDB7DEB79C
:1003E000880F880F880F806469837A830E94530185
:1003F00069817A81462F572F7A0118E0F7018191A0
:100400007F010E9443011150C9F70F900F90CF91C7
:10041000DF911F91FF90EF9008951F920F920FB6FA
:100420000F9211242F938F939F93EF93FF938BB190
:100430009CB1E0916500EF5FEF7120916400E217DD
:1004400041F08871E0936500F0E0E857FF4F90833A
:1004500001C082E08093A800FF91EF919F918F915E
:100460002F910F900FBE0F901F9018951F920F9213
:100470000FB60F9211248F939F93EF93FF93909158
:10048000660080916700981761F0E0916700EF5F68
:10049000EF71E0936700F0E0E859FF4F80818CB97D
:1004A00001C05598FF91EF919F918F910F900FBED2
:1004B0000F901F901895109266001092670010928E
:1004C00065001092640097FF03C022E02BB99F776C
:1004D00090BD89B988E98AB986E880BD0895909170
:1004E000650080916400981789F0E0916400EF5FE7
:1004F000EF71E0936400F0E0E857FF4F8081909146
:10050000A800392F20E0280F311D02C020E031E083
:10051000C9010895909166009F5F9F7120916700C7
:100520009217E1F3E92FF0E0E859FF4F80839093B1
:100530006600559A0895EF92FF92CF93DF93E82ECD
:10054000E7017E01F92EE70102C00E948A0289912B
:100550008823D9F7DF91CF91FF90EF900895CF9343
:10056000DF93EC0102C00E948A02FE012196849171
:100570008823C9F7DF91CF9108958091650020917C
:10058000640090E04F96821B91096FE170E00E9439
:10059000CF0208958091640080936500089597FBD1
:1005A000092E07260AD077FD04D00CD006D00020F3
:1005B0001AF4709561957F4F0895F6F7909581959F
:1005C0009F4F0895AA1BBB1B51E107C0AA1FBB1F69
:1005D000A617B70710F0A61BB70B881F991F5A95CF
:1005E000A9F780959095BC01CD010895F894FFCFAF
:00000001FF
